:100000000AC018951895189518951895189518956B
:100010001895189518958FED8DBFC0ECE0EC4E2E1D
:10002000DD275D2EEEE7F0E0A0E6B0E088278D93B7
:100030003197E9F7A8D266248FE087BB80E088BBC0
:100040008FEF81BB80E082BB84E690E010D38CE030
:10005000E2D2BF98A7E69C9197FF04C0B7990EC063
:100060009F779C93B79B0AC088E29F939927FFD202
:100070009F91B79B03C090689C9314D26AD2E4EE20
:10008000F6E05FD264D2E4EFF6E05BD2E2E0F0E0CB
:1000900071D280E080936400A1E6FCD280E080937E
:1000A000630080E08093650054D2E4E0F7E049D239
:1000B0008FE087BB80E788BB8AE090E0D8D281E000
:1000C00080936000A6E30C9105FB81E00EF480E0D4
:1000D0008F93A6E30C9106FB81E00EF480E09F91E4
:1000E0008923882309F401C009D182E0809360004C
:1000F000A6E30C9104FB81E00EF480E08F93A6E36D
:100100000C9105FB81E00EF480E09F918923882308
:1001100009F401C0F3D083E080936000A6E30C9162
:1001200004FB81E00EF480E08F93A6E30C9106FBC4
:1001300081E00EF480E09F918923882309F401C0B7
:10014000DDD08FE187BB88E688BB8AE090E08FD264
:1001500084E080936000A6E30C9105FB81E00EF43F
:1001600080E08F93A6E30C9106FB81E00EF480E023
:100170009F918923882309F401C0C0D085E0809332
:100180006000A6E30C9105FB81E00EF480E08F9304
:10019000A6E30C9106FB81E00EF080E09F9189239D
:1001A000882309F401C0AAD086E080936000A6E30A
:1001B0000C9105FB81E00EF080E08F93A6E30C919B
:1001C00006FB81E00EF480E09F918923882309F4E7
:1001D00001C094D08FE287BB88E588BB8AE090E0BD
:1001E00046D287E080936000A6E30C9104FB81E097
:1001F0000EF080E08F93A6E30C9106FB81E00EF4F5
:1002000080E09F918923882309F401C077D088E09A
:1002100080936000A6E30C9104FB81E00EF480E083
:100220008F93A6E30C9106FB81E00EF080E09F9196
:100230008923882309F401C061D089E0809360009C
:10024000A6E30C9104FB81E00EF480E08F93A6E31B
:100250000C9106FB81E00EF480E09F9189238823B6
:1002600009F401C04BD08FE487BB88E388BB8AE0E8
:1002700090E0FDD18BE080936000A6E30C9104FB3D
:1002800081E00EF080E08F93A6E30C9105FB81E006
:100290000EF480E09F918923882309F401C02ED0B9
:1002A0008AE080936000A6E30C9104FB81E00EF4E9
:1002B00080E08F93A6E30C9105FB81E00EF480E0D3
:1002C0009F918923882309F401C018D08CE0809382
:1002D0006000A6E30C9104FB81E00EF480E08F93B4
:1002E000A6E30C9105FB81E00EF080E09F9189234D
:1002F000882309F401C002D0DBCEA6CE939A84E60F
:1003000090E0B5D1939884E690E0B1D1009164007B
:10031000013009F001C02AC000916400023009F0E8
:1003200001C047C0009160000B3009F00CC011D132
:10033000E2E1F7E006D1A4E68C918F5F8C9380E038
:1003400080936300B5CE009160000C3009F00DC0C1
:10035000EAE0F0E0A4E1BED1A1E60D911C91041702
:10036000150709F001C088C065C036C00091600063
:100370000C3009F01DC0EAE0F0E0A4E1ABD1A1E649
:100380000D911C910417150709F401C053C0A1E693
:1003900081D180E08093630080E080936500A4E6D3
:1003A0008C918F5F8C93D5D0E2E2F7E0CAD080CEFB
:1003B00013C0009160000C3009F00EC0EAE0F0E0DC
:1003C000A1E67BE776D1C5D0E2E3F7E0BAD043D02F
:1003D000E2E0F0E0CFD05DCEA3E68C918F5F8C930E
:1003E0000091630046E0040FA5E60C938FEBA5E6B1
:1003F0001C91BED0E2E4F7E0A4D000916300043089
:1004000010F009F001C001C015C0A1E60D911C91CA
:100410004AE050E083D0A1E60D931C93A1E60D9134
:100420001C91A0E64D915527040F151FA1E60D93D1
:100430001C9308958ED0E4E4F7E083D0939AE3E030
:10044000F0E098D0939883D0E4EEF6E07AD0E4E13F
:10045000F0E090D01ECE84E690E009D1939A88EC2B
:1004600090E005D1939888EC90E001D1939A88ECC4
:1004700090E0FDD0939808956CD0E2E3F7E061D06E
:10048000EADF65D0E2E5F7E05CD08CE291E0EFD006
:10049000949AE1E0F0E06ED094985BD0E1E0F0E077
:1004A00069D0F7CDE1E0F0E065D0B79901C014C0A4
:1004B000EAE0F0E002ED14E0A0E1BB277BE7F9D031
:1004C000CADF47D0E0E6F7E03CD041D0E0E7F7E014
:1004D00038D0E5E0F0E04ED0089504D01FD000FC05
:1004E0000CD008950024E89457FF02C009D0689406
:1004F00000F80BD010F80124089502D009D0089517
:10050000509540954F5F5F4F0895E89417FF089509
:10051000009510950F5F1F4F68940895752F642FF5
:1005200055274427FF93F1E1889405C010F4460F46
:10053000571F5695479517950795FA95B9F7FF9167
:100540000895A4D0802D11F060D0FBCF089580ECE9
:1005500062C081E060D014D080E85DC08FE72130B8
:1005600039F08FEB223021F08FE8233009F08FEC47
:10057000810F51C088EE93E07AD03197D9F7089572
:1005800083E0992774C08AEF90E071D0BB9ABA9A41
:10059000B99AB89A8E9A8D9A959885E090E067D02E
:1005A0009698C398C298C19AC09A969AEF93FF936F
:1005B000E0E6F0E050D0FF91EF91969855D0969AF2
:1005C000EF93FF93E0E6F0E046D0FF91EF9196982D
:1005D0004BD0969AEF93FF93E0E6F0E03CD0FF918A
:1005E000EF91969841D0C098969AEF93FF93E0E6EA
:1005F000F0E031D0FF91EF91969836D088E20BD0A1
:100600008EE009D086E007D00895959A829505D0AE
:1006100004D02AD008959598F9CF859510F4C09A02
:1006200001C0C098859510F4C19A01C0C198859504
:1006300010F4C29A01C0C298859510F4C39A01C003
:10064000C398969AEF93FF93E0E6F0E004D0FF9111
:10065000EF91969808953197F1F70895689462F8AC
:100660000895E89462F8089581E090E000C0EF9367
:10067000FF93EE27E82BE92B31F0E8EEF3E031971A
:10068000F1F70197D1F7FF91EF910895C895319651
:100690000020089582E001C084E099279D938A9507
:1006A000E9F70895E199FECFEEBB3196089591E008
:1006B00001C092E07B3751F47FB7F894F3DF8D915E
:1006C0008DBBE29AE19A9A95C9F77FBF7727089583
:1006D00091E001C092E0E6DFE09A8DB38D939A95A8
:1006E000D1F708955757572E4156522E344D472E65
:1006F000434F4D00436F64654C6F636B415652200E
:100700002D205200202020456E74657220636F6496
:10071000650020456E746572206F6C6420636F64A1
:10072000650020456E746572206E657720636F6486
:10073000650020436F646520616363657074656460
:1007400000002A00202020436F64652077726F6EBE
:10075000670020202020556E6C6F636B656400007D
:100760002020496E697469616C20636F64650000C4
:1007700020202020206973202020313233340000D3
:00000001FF
